:020000040000FA
:06080000D5EF04F0120028
:0608080029EF04F01200CC
:0608180016EF04F01200CF
:02082A000000CC
:04082C00D8CFE4FF3E
:10083000E0CFE4FFE46EDACFE4FFE2CFDAFFE65286
:10084000E552E5CFDAFFE550E5CFE0FFE5CFD8FF91
:100850001000DACFE4FFE2CFDAFFE652E552E5CF4F
:10086000DAFF1100896A92680F0EC16E070EB46E2E
:100870008A6A93688B6A9468FC0E8B16FC0E941639
:1008800094848B808B82C80EE66EBEEC04F0E55239
:10089000C80EE66EBEEC04F0E552C80EE66EBEEC85
:1008A00004F0E552C80EE66EBEEC04F0E5528B9003
:1008B0008B92C80EE66EBEEC04F0E552C80EE66EF2
:1008C000BEEC04F0E552C80EE66EBEEC04F0E55254
:0E08D000C80EE66EBEEC04F0E552D3D712005F
:0208DE002A0EE0
:1008E000F66E080EF76E000EF86E00010900F55066
:1008F000656F0900F550666F03E1656701D03DD073
:100900000900F550606F0900F550616F0900F5505E
:10091000626F09000900F550E96E0900F550EA6EB2
:10092000090009000900F550636F0900F550646F74
:1009300009000900F6CF67F0F7CF68F0F8CF69F04B
:1009400060C0F6FF61C0F7FF62C0F8FF00016353AB
:1009500002E1645307E00900F550EE6E6307F8E228
:100960006407F9D767C0F6FF68C0F7FF69C0F8FFF2
:0C09700000016507000E665BBFD7120097
:04097C00FF0EE35037
:10098000036EEF0E01D0F30EE76EE72EC5EF04F015
:100990000C0E026EE76AE72ECBEF04F0022ECAEFD0
:0A09A00004F0032EC3EF04F0120070
:0609AA0013EE00F023EE45
:1009B00000F0F86A019C6FEC04F032EC04F0FDD713
:0209C000120023
:0E09C20000EE00F00F0EEE6AEA62FDD71200A2
:00000001FF
